:100000000C945C000C946E000C946E000C946E00CA
:100010000C946E000C946E000C946E000C946E00A8
:100020000C946E000C946E000C946E000C946E0098
:100030000C946E000C946E000C946E000C946E0088
:100040000C9416010C946E000C946E000C946E00CF
:100050000C946E000C946E000C946E000C946E0068
:100060000C946E000C946E00000000002400270029
:100070002A0000000000250028002B0004040404CE
:100080000404040402020202020203030303030342
:10009000010204081020408001020408102001021F
:1000A00004081020000000080002010000030407FB
:1000B000000000000000000011241FBECFEFD8E0B8
:1000C000DEBFCDBF21E0A0E0B1E001C01D92A930AC
:1000D000B207E1F70E9460010C94CF010C9400007C
:1000E000E6EAF0E09491E2E9F0E02491EEE7F0E056
:1000F000E491EE2309F43CC0992339F1933091F057
:1001000038F49130A9F0923001F594B59F7D12C07A
:10011000973091F09830A1F09430B9F4909180002C
:100120009F7D03C0909180009F77909380000DC0C9
:1001300094B59F7794BD09C09091B0009F7703C09C
:100140009091B0009F7D9093B000F0E0EE0FFF1F04
:10015000EE58FF4FA591B4919FB7F894811104C058
:100160008C912095282302C0EC912E2B2C939FBFBD
:1001700008953FB7F8948091050190910601A091F0
:100180000701B091080126B5A89B05C02F3F19F0C3
:100190000196A11DB11D3FBFBA2FA92F982F882707
:1001A000820F911DA11DB11DBC01CD0142E0660F62
:1001B000771F881F991F4A95D1F708958F929F92B4
:1001C000AF92BF92CF92DF92EF92FF920E94B9005E
:1001D0004B015C0188EEC82E83E0D82EE12CF12C77
:1001E0000E94B900DC01CB0188199909AA09BB0951
:1001F000883E9340A105B10598F321E0C21AD108C9
:10020000E108F10888EE880E83E0981EA11CB11C5D
:10021000C114D104E104F10419F7FF90EF90DF90CD
:10022000CF90BF90AF909F908F9008951F920F92A4
:100230000FB60F9211242F933F938F939F93AF93F9
:10024000BF938091010190910201A0910301B091AF
:1002500004013091000123E0230F2D3720F4019693
:10026000A11DB11D05C026E8230F0296A11DB11DD9
:10027000209300018093010190930201A093030158
:10028000B09304018091050190910601A0910701AE
:10029000B09108010196A11DB11D809305019093B5
:1002A0000601A0930701B0930801BF91AF919F9100
:1002B0008F913F912F910F900FBE0F901F90189527
:1002C000789484B5826084BD84B5816084BD85B531
:1002D000826085BD85B5816085BD80916E0081603D
:1002E00080936E00109281008091810082608093E3
:1002F00081008091810081608093810080918000E5
:100300008160809380008091B10084608093B1000F
:100310008091B00081608093B00080917A00846009
:1003200080937A0080917A00826080937A00809135
:100330007A00816080937A0080917A00806880934F
:100340007A001092C100E2E9F0E02491EEE7F0E0DB
:100350008491882399F090E0880F991FFC01E85957
:10036000FF4FA591B491FC01EE58FF4F85919491F8
:100370008FB7F894EC91E22BEC938FBFC0E0D0E004
:1003800081E00E9470000E94DE0080E00E94700008
:100390000E94DE002097A1F30E940000F1CFF894A4
:0203A000FFCF8D
:00000001FF
